:020000040800F2
:10500000381F0020D5500008B99200087F89000899
:105010000000000000000000000000000000000090
:105020000000000000000000000000000D970008D4
:10503000000000000000000035930008B997000848
:10504000E7500008E7500008E7500008E750000864
:10505000E75000085D5C0008E7500008E7500008D2
:1050600000000000E7500008655B0008E7500008FA
:10507000E7500008D58D000800000000E750000848
:1050800000000000E75000080000000000000000E1
:10509000E750000800000000E7500008E750000853
:1050A000E7500008E7500008E750000891A6000804
:1050B000E7500008E7500008000000000000000072
:1050C0000348854600F098FC0048004785B6000874
:1050D000381F00200448804704480047FEE7FEE7E9
:1050E000FEE7FEE7FEE7FEE779980008C1500008FA
:1050F00030B50B46014600202022012409E00D4670
:10510000D5409D4205D31D469540491B25469540F7
:1051100040191546521E002DF1DC30BD70B500243B
:105120002546002801DA01244042002901DA012540
:105130004942FFF7DDFFAC4200D04042002C00D0D6
:10514000494270BDF0B51FB40646002082B0054646
:105150004024019100901BE0019922460F46304601
:1051600000F086FB049A059B801A994110D31046E3
:105170001946224600F06CFB361A8F4101972246F1
:1051800001200021009F00F063FB38184D41009082
:105190002046641E0028DFDC019B00982946324629
:1051A00007B0F0BD03460B439B0703D009E008C9D5
:1051B000121F08C0042AFAD203E00B780370401CC7
:1051C000491C521EF9D27047D2B201E00270401C55
:1051D000491EFBD270470022F6E710B513460A4677
:1051E00004461946FFF7F0FF204610BD30B50446CF
:1051F0000020034600E05B1C934203D2E05CCD5CE0
:10520000401BF8D030BDF8B502464A40D40F4200EA
:105210004B0052085B089A4202D2024608461146E9
:105220004A0023D0C30D4A00DDB2120EAD1A202D64
:1052300035DA49020126490AF6058A19002C00D000
:10524000524220214F1B1146B9402A411018C20D6D
:105250009A4221D0002C17D0012D08DCDA05801AE3
:10526000D20F8019D207DBB200F02EFBF8BDDA05B1
:10527000801A012340001B06C01880185A4280186B
:10528000CA0F1043490007E04908C2071143DA0575
:10529000801A80194008801800F00EFBF8BD6100EC
:1052A0000122511A001BF7E70122D2075140AAE759
:1052B0000122D2075040A6E7024670B54A40D30FFC
:1052C000DB0740002DD04A002AD0010E140E000248
:1052D00012020919400A520A8418E501044654438F
:1052E000000A120A2E045043A4194219200CC54387
:1052F000AA18120C0125AD03521C521912047F3951
:10530000240400D0521C104301D44000491EC2B2F4
:105310000C06C0092018401C4008802A02D003E077
:10532000002070BD40084000002900DA002018432A
:1053300070BD70B502464A40D50F40004A00ED07E7
:1053400040085208002814D0002A12D0C40DD30DF2
:1053500041020120C0055202490A520AE41A091802
:1053600012187D34914201D3641C00E04900002CE6
:1053700001DA002070BD0023914201D3891A034352
:10538000400849000028F7D100290AD0914202D1F3
:105390000121C90705E0914201D2012101E001216B
:1053A000C943E005C018401900F086FA70BD00003E
:1053B000F0B507460846584087B0C00F0490480033
:1053C0000E46590040084908BC1A884105D23846A3
:1053D00031461E4617460B46024658004008104309
:1053E0004CD0300D039040055900400D490D0590FB
:1053F000401A0290402872DA18030121000B0905B7
:105400000843019004980092002805D00199524267
:105410000020884100920190029840210A1A0199C7
:10542000009800F015FA05460C466B4607CB00F0D5
:1054300030FAC0197141039A0E0D0023D717564058
:105440001A467A40164344D0049A002A2DD0029A74
:10545000012A039A15DC1205C01A9141012636056E
:10546000001C7141D20F059ED20700930192029653
:105470002A46234600F06EFA07B0F0BD38463146A2
:10548000FAE71605224A0F46B218C01AB7410121A1
:105490000905001C4F4100187F4111461818794139
:1054A000E20F10436D19644113E0E2076D081543E4
:1054B0006408C2071443039A01261205C01A9141D9
:1054C0003605001C7141CE07400830434908C0181A
:1054D00051412A46234600F030FACDE7FFE7049811
:1054E00001224000C117121A00238B410498314653
:1054F000C417381AA141EEE730B40124E407634031
:1055000030BC55E730B40124E407614030BC4FE7BC
:105510000000E0FFF0B51FB488B00B990998002493
:1055200048400999C00F490049080991C0070B99E3
:105530000090490049080B9109990898A64608432C
:105540001CD00B990A98084318D0099801244000F0
:10555000420D4800410D099824050003000B20432B
:1055600009900B980003000B20430B9050181C4926
:105570004018002201901446104605E00020014624
:105580000DB0F0BD032801DA034600E003239C467A
:10559000C11A0AAE0AE05F0008ADED5B4F00F75B91
:1055A0007D430027AA187C41491C5B1E6145F2DD42
:1055B000410004AB5A522104120C0A43240C401C33
:1055C0000828DFDB01980290009970460191009055
:1055D000059B049A0799069800F0BCF9D0E70000F3
:1055E0000DFCFFFFF0B50C465C4085B0E40FE4070E
:1055F00003944C000026640859009446490802466A
:105600000296224321D062460A431ED06200570D03
:105610004A000E032303550D012402462C4924059C
:10562000781B1B0B360B4018234326436146009022
:105630001C46501AB44103D30098401C009002E06D
:10564000921800985B41002803DA0020014605B05B
:10565000F0BD0020012109050746864611E0644699
:105660001D46141BB54106D36546521BB341744613
:1056700007430C43A646CD07400849082843921823
:105680005B4105460D43EAD11046184313D06046EE
:10569000194650407140084306D06046101AB34185
:1056A00006D20122002306E000220123DB0702E0EC
:1056B0000122D2435310009874460105381C614101
:1056C000029C039D0019694100F037F9BFE7000013
:1056D000FD030000C217C10F504010B54018CA07A3
:1056E0009623002100F0F0F810BD10B5002296239B
:1056F000114600F0E9F810BD0EB5C217C10F5040B9
:10570000CA0740180021054B0293019200910A46F6
:105710000B4600F01FF903B000BD00003304000089
:105720000EB505490291002100910A460B460191F0
:1057300000F010F903B000BD330400004100400246
:105740000122400AD205090E80187F2901DA0020C3
:105750007047962903DC9622511AC8407047963943
:10576000884070474A0009030123090B1B051943B0
:10577000094B10B5520D9A4201DA002010BD064BBC
:1057800034339A4203DC9A1A00F072F810BD0349D0
:105790005118884010BD0000FF030000CDFBFFFF43
:1057A000C20FD207400040080BD0C10D0723DB0118
:1057B000C91840020905400A1143C20840071143B5
:1057C000704700200146704710B5002904DB012412
:1057D000E40740428C412146002B04DB1C46012398
:1057E000DB075242A341994200D1904210BD000014
:1057F000CB0FDB07490010B5490802460A4307D022
:105800000A0D07240903E401090B121B002A01DC1D
:10581000002010BDC900440F0C43C100E018D205A0
:10582000801800F049F810BD0122D207002800DBE3
:10583000101A002900DB511A814270470122D20759
:10584000002800DB101A002900DB511A884270473B
:1058500010B5202A04DB0146203A9140002010BDFB
:10586000914020239C1A0346E3401943904010BD09
:1058700010B5202A04DB0846203AD040002110BD94
:105880000B46D340D0402024A21A91400843194629
:1058900010BD10B5202A06DBCB170846203A104170
:1058A000C1170B4306E00B461341D0402024A21A37
:1058B00091400843194610BD002904DA401C4900F4
:1058C00001D140084000704770B40024050C05D198
:1058D0001024000402D1002921D01124050E01D189
:1058E00000020834050F01D10001241D850F01D1EC
:1058F0008000A41C002801DB4000641C002908D0A3
:1059000020252E1B0D46F540A14000D00121294342
:10591000084301061B1B000ADB1D02D5002070BCDA
:105920007047DB05181880180029F8DA401C490078
:10593000F5D170BC40084000704710B5002B08DA64
:105940000024401C614192185B411A4301D1400878
:10595000400010BDF0B51FB482B005460C0003D066
:10596000084604F0A5FF02E004F0A2FF2030024642
:10597000009021462846FFF76BFF049B059A0446DA
:105980000F4618431143084314D0184610431BD048
:10599000009840210A1A18460599FFF769FF054645
:1059A0000E46009A05990498FFF752FF084305D068
:1059B000012004E02046394607B0F0BD0020C117A1
:1059C00005430E432C43374300990E986305401A54
:1059D0007905E40A00220C43FD0A0A3002D50020B2
:1059E0000146E9E70105101969410C9C0D9D00195C
:1059F0006941FFF7A2FFDFE7064C0125064E05E0EF
:105A0000E36807CC2B430C3C98471034B442F7D3DF
:105A1000FFF75AFBE0B9000800BA000870B58C180F
:105A20000578401C6B075B0F01D10378401C2A11DD
:105A300006D10278401C03E006780E70401C491C19
:105A40005B1EF9D12B0705D40023521E0DD40B7019
:105A5000491CFAE70378401CCB1A921C03E01D781E
:105A60000D70491C5B1C521EF9D5A142D8D30020F1
:105A700070BD000038B50446074908480068FFF7C4
:105A800037FB6043009002E00098401E00900098B1
:105A90000028F9D138BD000040420F00500100201D
:105AA00070B504460025206880688007800F0128B3
:105AB00007D120680068C007C00F002801D001206E
:105AC00000E00020002839D1206880681C49084087
:105AD000002801D1012000E00020002809D1606DDC
:105AE000102108436065A06D01210843A0650120D5
:105AF00070BD20688068012108432168886001200A
:105B0000FFF7B8FF01F0ECF805460EE001F0E8F809
:105B1000401B0A2809D9606D102108436065A06DFB
:105B200001210843A0650120E2E720680068C00762
:105B3000C00F0121484048400028E7D00020D7E7A7
:105B40001700008010B502460B460020002103E03C
:105B5000545C2418A0B2491C9942F9D3C443A0B2A2
:105B600010BD000010B5034800F0B8FD024800F079
:105B7000B5FD10BDD81A0020901A002030B51C25A4
:105B8000446C2C400125A540046C6560046863608A
:105B90008468102C04D10468A2600468E16003E00A
:105BA0000468A1600468E26030BD000010B5012007
:105BB0001749487202201749487203201649487253
:105BC0000420164948721248154909780170124894
:105BD0001349097801700F481149097801700422AE
:105BE00010490B48401DFFF7DDFA04220D490A4811
:105BF000401DFFF7D7FA04220A490648401CFFF768
:105C0000D1FA042207490548401CFFF7CBFA10BD22
:105C100084150020BE150020A61500209815002030
:105C2000270100201C01002010B503F071FC20208A
:105C300003F0B0FD012005F02FFA002003F0AAFDCB
:105C4000044805F0BFF8044805F0A4FB002005F067
:105C5000E1FB10BD600000208380000010B5012131
:105C60000520000701F02CF8002802D000200A4986
:105C700008600221094801F023F8002805D10848EE
:105C800000880A21484307490880012000F012FFDC
:105C9000022000F00FFF10BD48010020000400505A
:105CA00036010020400100207047000000210A4A10
:105CB00051610A494968012252021143074A516061
:105CC0001146496808221143044A51600021C20963
:105CD000D201116070470000201B0020002002400C
:105CE0007FB504460D460020039000F09BFE002087
:105CF00000900194E809029003A9684600F014FEA0
:105D0000002804D000F056FE002004B070BD00F062
:105D100051FE0120F9E710B50346002002E01C5CAB
:105D20000C54401C9042FAD310BD000000203949A9
:105D30008969FF2201321140914208D136494969EF
:105D400002221143344A5161FF2101310843314994
:105D50008969012252021140914208D12E494969B4
:105D6000012211432C4A516101214902084329496A
:105D70008969012292021140914208D1264949695C
:105D800008221143244A5161012189020843214913
:105D900089690122D2021140914208D11E49496904
:105DA000042211431C4A51610121C90208431949C7
:105DB0008969012252031140914208D1164949696B
:105DC00010221143144A516101214903084311492A
:105DD0008969012252041140914207D10E49496953
:105DE000202211430C4A5161202108430949896945
:105DF000012212041140914208D107494969402209
:105E00001143054A51610121090408430149886190
:105E10007047000000200240201B002070B504469F
:105E200000F05EFF05460BE0601C002808D0002C47
:105E300004D000F055FF401BA04201D9032070BDE3
:105E40001F488069C007C00F0028EDD11C48806939
:105E500002210840022801D1194988611848806947
:105E6000FF2101310840884223D01548806949004C
:105E7000084088421DD01248806949000840884285
:105E800017D00F48806949000840884211D00C485B
:105E900080698900084088420BD00948806909015F
:105EA0000840884205D00648806949100840884269
:105EB00003D1FFF73BFF0120C1E70020BFE700004F
:105EC00000200240F0B585B006460F461446002576
:105ED000029601970020009000F0A4FD13E00198C5
:105EE000006803900220039A029900F073FD00906D
:105EF0000098002800D008E00298001D0290019848
:105F0000001D01902D1DA542E9D300BF00F052FDF8
:105F1000A54202D2002005B0F0BD0120FBE7000041
:105F200010B50B4800F070FB0A21094800F0F6FAA2
:105F3000074800F09DF9012149020840884204D138
:105F4000034800F098F980B210BD00BFFCE70000E4
:105F50002C190020F0B587B000220121404800F044
:105F6000B8FEFFF7DDFF0546FFF7BFFB04463D49DE
:105F7000FFF7DFF93C49086001221146384800F07C
:105F8000A8FE39480068FFF70BFC04460022374B97
:105F9000FFF71AFC5DD836480078002821D0002091
:105FA00033490870FFF7BCFF0546FFF79EFB044628
:105FB0002C49FFF7BEF92C49086008460068FFF736
:105FC000EFFB04460022294BFFF796FA0022294BEB
:105FD00005910490FFF79EFA0646FFF709FC264953
:105FE000086021480068FFF7DBFB064600221F4BD4
:105FF000FFF782FA0446214A214BFFF78BFA0391FF
:1060000002901D480068FFF7CBFB04461B4A524232
:106010001C4BFFF77FFA01910090039B029AFFF758
:10602000C7F905910490FFF7E3FB1349086016498F
:1060300011480068FFF702FC02D213480E490860BD
:1060400000210D480068FFF7EFFB02D200200A494B
:10605000086009480068FFF771FBC0B207B0F0BDE7
:106060000004005000401B442800002000000C40A9
:106070003000002000E064402C0000203333333334
:1060800033B33040CCCCEC3F0000C842F8B50446F6
:1060900000250026002700BF5020005D012801D107
:1060A0000220F8BD01215020015500BF2068806802
:1060B0008007800F012806D120680068084000286A
:1060C00001D0012000E00020002841D1606DFF21B7
:1060D000013188430221084360652068C068870752
:1060E000BF0F2068C068800880002168C8602068F1
:1060F00080680121C90708432168886000F0F0FD2D
:10610000064611E000F0ECFD801B0A280CD9606DFA
:106110000221884310210843606500BF0021502000
:10612000015500BF0120BCE720688068C00FC00790
:106130000121C9078842E5D02068C068384321683A
:10614000C860606D0221884301210843606504E056
:10615000606D202108436065012500BF00215020AB
:10616000015500BF28469CE770B504460D4600BFA8
:106170005020005D012801D1022070BD0121502076
:10618000015500BF2068806804210840800800286D
:106190000AD0606D20210843606500BF00215020B7
:1061A000015500BF0120E8E72D496868884229D0E1
:1061B0002068806A29684903490B0843216888627E
:1061C00028684003400B2749084001218904884280
:1061D00008D12548806849010843234988600A207E
:1061E000FFF748FC28684003400B20490840012184
:1061F000490488422CD11C488068490108431A4947
:10620000886025E02068806A29684903490B884333
:106210002168886228684003400B12490840012128
:106220008904884205D110488068490188430E4995
:10623000886028684003400B0C490840012149044C
:10624000884205D10848806849018843064988602A
:1062500000BF00215020015500BF00208DE7000045
:106260000110000000000448002701400000024423
:106270000146486D704701460868006C7047000091
:1062800010B50446002C01D1012010BD606D00281E
:1062900006D1A065002150200155204600F00EF9DE
:1062A000606D10210840102806D020688068042105
:1062B0000840800800280AD0606D102108436065FE
:1062C00000BF00215020015500BF0120DDE7606DB7
:1062D000FF210131884302210843606520688068FE
:1062E0008007800F012807D120680068C007C00F11
:1062F000002801D0012000E0002000283AD100BF92
:10630000032189076068884207D049426068884253
:1063100003D04900606888420CD120680069800081
:106320008008216808612068006961680843216865
:10633000086112E020680069800080082168086117
:106340005C4880680F21890488435A498860084660
:106350008068616808435749886000BF2068C0684A
:10636000182188432168C8602068C068A168084374
:106370002168C8604F4880680121490688434D491B
:10638000886008468068A18E4906084349498860AC
:1063900020688068012109070840002804D120688E
:1063A00080680843216888602068C06842490840C6
:1063B0002168C8602169E068022901D1042100E058
:1063C000002108432021095D490308432C21095D70
:1063D00049000843216B0843A16989030843E16927
:1063E000C90308432168C96808432168C860FF21C0
:1063F000C231606A884207D0A16A606A0843216896
:10640000C96808432168C8602120005D012813D1B4
:106410002020005D002807D12068C0680121090400
:1064200008432168C86007E0606D2021084360656B
:10643000A06D01210843A065E06B012817D12068F9
:106440000069FF218900884321680861216C606C24
:106450000843A16C08432168096908432168086161
:106460002068006901210843216808610BE0206869
:106470000069C007C00F002805D0206800694008E7
:1064800040002168086120684069C008C000216898
:10649000486120684069A16B084321684861002079
:1064A000A065606D022188430121084360650020DA
:1064B000EBE60000002701401902FEFF10B586B090
:1064C0000446142101A8FEF786FE1249206888427E
:1064D0001ED11148406B491508430F49486300BF5E
:1064E0000846C06A012108430B49C8620846C06AD1
:1064F000C007C00F009000BF00BF02200190032022
:1065000002900020039001A90520000700F0E2FAA4
:1065100006B010BD0024014000100240F8B504464A
:106520000D46002600276069082801D1082711E0E0
:106530002068C068C007C00F00280AD0606D202105
:106540000843606500BF00215020015500BF0120B5
:10655000F8BD0C2700F0C4FB064614E0681C0028B8
:1065600011D0002D04D000F0BBFB801BA8420AD93B
:10657000606D04210843606500BF00215020015573
:1065800000BF0320E4E72068006838400028E5D019
:10659000606D01214902084360652068C0680321DD
:1065A00089020840002826D12020005D002822D141
:1065B000206800680821084008281CD120688068ED
:1065C00004210840800800280DD1206840680C2173
:1065D000884321684860606DFF21013188430121B3
:1065E0000843606507E0606D202108436065A06D89
:1065F00001210843A065A069002802D10C20216870
:1066000008600020A4E7000070B50446002520685B
:10661000806804210840800800282BD100BF50204A
:10662000005D012801D1022070BD012150200155DB
:1066300000BFE069012803D02046FFF731FA054684
:10664000002D18D1606D0D490840FF21013108432C
:1066500060650020A06500BF00215020015500BFEB
:106660001C20216808602068806804210843216894
:10667000886000E002252846D6E70000FEF1FFFF13
:1066800070B5044600252520005D022803D00420B3
:10669000E063012520E0206800680E21884321681E
:1066A00008602068006840084000216808601C21DC
:1066B000606C084001218140206C4160012125204F
:1066C000015500BF00212420015500BFA06B002808
:1066D00002D02046A16B8847284670BD70B504469D
:1066E000206C0568206806681C20616C014004204D
:1066F0008840284000281DD004203040002819D0B0
:106700002068006820210840002805D12068006822
:1067100004218843216808601C21606C0840042122
:106720008140206C4160206B00285AD02046216BAC
:10673000884756E01C20616C0140022088402840B8
:10674000002825D002203040002821D02068006891
:1067500020210840002808D1206800680A218843C9
:10676000216808600121252001551C21606C08402A
:1067700002218140206C416000BF0021242001558E
:1067800000BFE06A00282CD02046E16A884728E054
:106790001C20616C0140082088402840002820D03F
:1067A0000820304000281CD0206800680E21884353
:1067B000216808601C21606C084001218140206C28
:1067C00041600120E06301212520015500BF002127
:1067D0002420015500BF606B002802D02046616B69
:1067E000884770BD70B50446002C01D1012070BDF2
:1067F000244A2168881A1421FEF77AFC800060641C
:1068000020480838206402212520015520680568A9
:106810001D480540E168A068084321690843616993
:106820000843A1690843E1690843216A0843054315
:106830002068056001218903A068884217D01148AB
:106840007830806A1C22616C11400F228A4090438C
:106850000C49783188621C22616C11406068884064
:1068600008497831896A08430649783188620020EE
:10687000E06301212520015500212420015500203D
:10688000B5E70000080002400F80FFFFF8B504469E
:106890000D4616461F460020009000BF2420005DD4
:1068A000012801D10220F8BD01212420015500BF9B
:1068B0002520005D01282DD1022125200155002031
:1068C000E0632068006840084000216808603B469B
:1068D000324629462046FFF751F9206B002806D0A2
:1068E000206800680E210843216808600BE02068DA
:1068F00000680421884321680860206800680A2134
:106900000843216808602068006801210843216865
:10691000086006E000BF00212420015500BF0220CE
:1069200000900098BFE70000F8B504460E46012726
:10693000002500BF1C48007C012801D10220F8BDC1
:1069400001201949087400BF1848FFF767FA074685
:10695000002F22D1401E3060656817E02846FFF7FF
:10696000A5F91248FFF75AFA07461148406808216E
:1069700088430F49486008464068491588430C49D8
:106980004860002F01D0356006E08035A068C00166
:1069900061684018A842E1D800BF00BF002002494A
:1069A000087400BF3846CAE7201B002050C300000F
:1069B000002002400648406802210843044948601C
:1069C000084640680121084301494860002070479B
:1069D00000200240F8B507460C461546012600BFC8
:1069E0000E48007C012801D10220F8BD01200B498E
:1069F000087400BF0A48FFF711FA0646002E06D1B8
:106A00000649486125600648FFF708FA064600BFB8
:106A100000200249087400BF3046E6E7201B002032
:106A200050C300001D484068C007C00F002816D0A2
:106A300000BFEFF31080014600BF72B61848174A36
:106A4000D0601848D06000BF81F3108800BF1046A6
:106A50004068C007C00F002801D0012070470F48D0
:106A6000406802221040022815D100BFEFF31080C9
:106A7000014672B60C48094A10610C48106108467C
:106A800080F3108800BF10464068022210400228A0
:106A900001D10120E2E70020E0E7000000200240F1
:106AA000EFCDAB8905040302BFAE9D8C1615141300
:106AB0007047000010B50446054840692040002892
:106AC00004D0034844612046FFF7F2FF10BD0000E8
:106AD0000004014070B50346002200240020DAE0E3
:106AE000012696400D6835402C46002C77D04D6825
:106AF000022D02D04D68122D15D1D508AE001D46CD
:106B00002035A8595507EE0E0F25B5400646AE4371
:106B100030465607F60E0D69B5402843D508AD003E
:106B20001E46203670514D68012D08D04D68022D4B
:106B300005D04D68112D02D04D68122D18D19868DE
:106B400056000325B5400646AE4330465600CD6894
:106B5000B540284398605868012595400646AE43E5
:106B6000304610264D6835402D0995402843586021
:106B7000186856000325B5400646AE4330460D79E9
:106B8000AD07AD0F5600B54028431860D8685600D1
:106B90000325B5400646AE43304656008D68B540E5
:106BA0002843D860012636074D683540B54271D17B
:106BB0003C4D6D6B012635433A4E75633A4D960850
:106BC000B600A85995072E0F0F25B5400646AE43CF
:106BD000304605252D07AB4202D1002515E059E0CE
:106BE000324DAB4201D101250FE0314DAB4201D115
:106BF00002250AE02F4DAB4201D1032505E02E4DC1
:106C0000AB4201D1052500E006259607360FB540B9
:106C10002843254D9608B600A851284D28680546FA
:106C2000A5432846012636044D683540B54202D1B9
:106C3000054625432846214D286068680546A5433A
:106C40002846012676044D683540B54202D10546F6
:106C500025432846194D6860A8680546A54328467F
:106C6000012636054D683540B54202D1054625431B
:106C70002846124DA860E8680546A5432846012627
:106C800076054D683540B54202D105462543284674
:106C90000A4DE860521C0D68D540002D00D01FE75A
:106CA00070BD0000001002400800014000040050C8
:106CB00000080050000C0050001C0050000401406F
:106CC000024613690B40002B01D0012000E0002098
:106CD0007047002A01D0816100E0816270470000A6
:106CE00001480068704700004C010020024800681D
:106CF000401C0149086070474C01002010B5002479
:106D0000084800684021084306490860002000F058
:106D10000BF8002801D0012401E000F0E1F9204641
:106D200010BD00000020024070B5044600257D2102
:106D3000C90009480068FEF7DBF9064601F066FB6A
:106D4000002801D0012504E000222146501E00F059
:106D5000EFF9284670BD00005001002070477047D1
:106D600070B505461F480078401C1E490870012078
:106D70001D4908701D4800881D49098840181B4995
:106D80000880084600881B49884203DD1A480088AD
:106D9000164908801548008818490968486118494B
:106DA000C888FEF7A2FC06461649FEF7C2FA04465A
:106DB000154801682046FEF726FA13490860104975
:106DC000488FFEF792FC04460F4801682046FEF704
:106DD0002BFD05D20D480078002801D004F0CEFC30
:106DE00070BD000046010020E600002030010020B8
:106DF0003201002029810000340100208819002080
:106E0000840D002000007A44480100203801002051
:106E1000704710B50446002C01D1012010BD02219D
:106E20002E200155204601F0DDFF204600F0F4F849
:106E300000212E20015500BF2D20015500BF00204C
:106E4000ECE77047704710B5044620680068C0073B
:106E5000C00F01214840484000280CD020688068BD
:106E6000084048404840002805D00120216848607B
:106E70002046FFF775FF206800680221084040089F
:106E800000280BD02068806808404008002805D002
:106E90000220216848602046FFF760FF20680068F4
:106EA00004210840800800280BD020688068084032
:106EB0008008002805D0042021684860204600F0A2
:106EC0000DF92068006808210840C00800280BD090
:106ED000206880680840C008002805D00820216884
:106EE00048602046FFF794FF2068006810210840A2
:106EF000000900280BD0206880680840000900289D
:106F000005D01020216848602046FFF728FF206840
:106F1000006820210840400900280BD020688068C4
:106F200008404009002805D02020216848602046FC
:106F3000FFF788FF2068006840210840800900288A
:106F40000BD02068806808408009002805D04020C8
:106F5000216848602046FFF774FF10BD70B50446F5
:106F6000002C01D1012070BD6068012800D100BF54
:106F700026496069884200D000BF2E20005D0028AD
:106F800005D100212D200155204600F059F802219D
:106F90002E2001552068C5686068012803D0890546
:106FA000A06A884203D11E21284688430546174916
:106FB0006069884201D01648054016480540A1681E
:106FC00060680843216A0843616A0843A16A08436C
:106FD00005436068012804D00121C905A06A8842E0
:106FE00003D1E16820690843054308496069884284
:106FF00005D06169A0690843E16908430543206839
:10700000C56001212E2001550020ACE7FFFF0000E4
:107010003F1FFFFFF8F119FF10B50446064920682D
:10702000884208D10548806B4000400803498863C6
:107030000D2000F065F810BD007C004000100240FB
:1070400010B504460949206888420DD10848806B74
:107050004905084306498863002201210D2000F0FC
:1070600067F80D2000F058F810BD0000007C0040CB
:107070000010024001460868C069704710B5034619
:1070800002242E20C4541448006824072043124CC4
:1070900020601868C0680124E40420431C68E06094
:1070A00018688068012420431C68A0601868006983
:1070B000012420431C6820611868816118684261BE
:1070C00018680069042420431C68206101242E20D4
:1070D000C454002010BD00000004014070470000AF
:1070E0000648406B01210843044948630846806B09
:1070F00009040843014988637047000000100240FA
:1071000000BFC206D20E01219140024A116000BFA9
:107110007047000080E100E000BFC206D20E0121EE
:107120009140024A116000BF7047000000E100E09A
:1071300070B504460D4616462946204602F0BEF8B4
:1071400070BD0000024949688143014A516070479F
:107150000070004003480068FF21013108430149E5
:107160000860704700700040024949680143014AC5
:1071700051607047007000400748006802210843D2
:10718000054908600548006904210843034908616E
:1071900000BF00BF30BF70470070004000ED00E04E
:1071A00010B5024600200E4B186880088000034688
:1071B000134318460A4B18600A4B1B6904242343E7
:1071C000084C2361012901D130BF02E040BF20BF3C
:1071D00020BF044B1B690424A343024C236110BD50
:1071E0000070004000ED00E0F8B504462021206862
:1071F000084020287CD120680840202800D100BF0A
:1072000000278148806B012109070840002805D12B
:107210007D48806B08437C49886301277B48006870
:10722000FF2101310840002816D178480068084342
:1072300076490860FFF754FD064606E0FFF750FD6B
:10724000801B642801D90320F8BD70480068FF2125
:10725000013108400028F1D06B4805680321090579
:107260000D4060680840A8420DD0091160680840D0
:10727000884208D1644800680121490408408842D6
:1072800001D10120E0E76048403000690321090492
:1072900008400546002D3DD060680840A84239D01E
:1072A000202120680840202834D157484030006908
:1072B00003210904884305465348403000690121F1
:1072C000C90408435049403108610846006901215A
:1072D000C90488434C49403108610846056180155E
:1072E00028408915884215D1FFF7FAFC064608E0C8
:1072F00039E0FFF7F5FC801B4549884201D903209E
:10730000A2E7414840300069012149020840400A93
:107310000028EED000BF00BF0321090460680840C8
:1073200088420AD1384800680901884303221205BF
:107330006168114008433449086000BF324840305A
:107340000069032212046168114008432E4940314C
:10735000086100BF012F05D12B48806B8905884348
:107360002949886300BF2078C007C00F002809D0D2
:1073700025484030C06880088000A1680843224941
:107380004031C860022120680840022809D11E4807
:107390004030C0680C218843E16808431A494031F5
:1073A000C86004212068084004280AD116484030EB
:1073B000C06803218902884321690843124940318A
:1073C000C86008212068084008280AD10E484030CB
:1073D000C068032109038843616908430A494031B1
:1073E000C86080212068084080280AD106484030C3
:1073F000C068032189048843A169084302494031D8
:10740000C860002020E7000000100240007000402B
:1074100088130000F8B504460D46002C01D1012068
:10742000F8BD79480068C007C00FA8420ED2764860
:107430000068400840002843734908600846006817
:10744000C007C00FA84201D00120E9E7022120684F
:107450000840022807D16D48C068F0218843A16820
:1074600008436A49C8602078C007C00F00284CD084
:107470006068022809D16548006801214904084074
:10748000400C002824D10120CAE76068032809D1F4
:107490005E480068012149060840400E002817D1C7
:1074A0000120BDE76068012808D158480068042120
:1074B0000840800800280BD10120B1E7534800683C
:1074C000012149020840400A002801D10120A7E714
:1074D0004E48C06880088000616808434B49C86016
:1074E000FFF7FEFB0646606802280FD107E0FFF7B2
:1074F000F7FB801B4649884201D9032090E74348A7
:10750000C0680C2108400828F1D134E060680328E5
:107510000FD107E0FFF7E4FB801B3D49884201D90A
:1075200003207DE73948C0680C2108400C28F1D1C0
:1075300021E0606801280FD107E0FFF7D1FB801B35
:107540003349884201D903206AE73048C0680C21DA
:1075500008400428F1D10EE007E0FFF7C1FB801BD3
:107560002B49884201D903205AE72848C0680C21DA
:1075700008400028F1D124480068C007C00FA84285
:107580000ED9214800684008400028431E49086081
:1075900008460068C007C00FA84201D001203FE79D
:1075A000042120680840042808D11848C068072131
:1075B00009028843E16808431449C860082120682B
:1075C0000840082809D11148C0680721C90288432A
:1075D0002169C90008430D49C86000F049F80B490A
:1075E000C968F022114009090A4A515CC8400A4999
:1075F00008600020FFF798FB0746002F01D03846AF
:107600000EE700200CE700000020024000100240BE
:1076100088130000BEB9000850010020014800682E
:10762000704700005001002000B5FFF7F7FF054943
:10763000C968072212021140090A034A515CC84076
:1076400000BD000000100240CEB9000800B5FFF7F1
:10765000E5FF0549C9680722D2021140C90A034A59
:10766000515CC84000BD000000100240CEB90008C7
:10767000FEB52E48C7680C203840002845D00428A5
:1076800004D008280CD00C283ED10BE02748006815
:1076900010210840002801D0254C00E0254C41E095
:1076A000254C3FE00F2080043840800C23490E5CBD
:1076B000032080053840800D401C01901B48C068A5
:1076C000012109040840002807D01B4971430846DE
:1076D0000199FDF70DFD054614E0144800681021DE
:1076E0000840002807D01249714308460199FDF768
:1076F000FFFC054606E00F49714308460199FDF776
:10770000F7FC05462C460DE000BF084840680721FD
:1077100049030840400B00900098401C0121814023
:10772000CC0300BF00BF2046FEBD00000010024099
:1077300000093D000024F40000127A00D6B90008C8
:10774000FEB50446002C01D10120FEBDF848C668F4
:107750000C210E40C768012109040F402078C007A2
:10776000C00F002872D0082E04D00C2E0FD108466E
:1077700087420CD1EE480068012149040840400CC2
:10778000002863D06068002860D10120DDE700BFD9
:10779000012109046068884205D1E5480068084372
:1077A000E349086027E005210904606888420ED19A
:1077B000DF480068012189040843DD490860084664
:1077C0000068012109040843D949086013E0D8483A
:1077D0000068012109048843D5490860084600680B
:1077E000012109040840009000BFD14800688900C9
:1077F0008843CF49086000BF6068002813D0FFF7B6
:107800006FFA054606E0FFF76BFA401B642801D9C2
:1078100003209AE7C6480068012149040840400C4B
:107820000028F0D012E0FFF75BFA054606E0FFF70C
:1078300057FA401B642801D9032086E7BC4800683A
:10784000012149040840400C0028F0D102212068A1
:10785000084002287AD1E0680290042E03D00C2E52
:1078600034D1002F32D1B24800680421084080088A
:10787000002804D00298002801D1012065E7AC4817
:1078800040681F2109028843216909020843A84969
:107890004860084600680921884302990843A449C2
:1078A0000860FFF7E5FEA249C968F0221140090906
:1078B000A04A515CC840A04908600020FFF734FA94
:1078C00001900198002841D001983EE702980028D5
:1078D00024D09748006809218843029908439449B5
:1078E0000860FFF7FDF9054606E0FFF7F9F9401BD0
:1078F000022801D9032028E78D48006804210840A8
:1079000080080028F1D08A4840681F210902884376
:107910002169090208438649486017E084480068E5
:107920004008400082490860FFF7DAF9054606E0A2
:10793000FFF7D6F9401B022801D9032005E77C4850
:1079400000680421084080080028F1D11021206837
:107950000840102867D1002E36D1754800684901CB
:107960000840400A002804D0A069002801D1012065
:10797000EBE66F484068072149038843216A0843C2
:107980006B494860084640680002000A217F0906EA
:10799000084367494860206A400B401C0121814030
:1079A000C8036349C968F02211400909614A515C62
:1079B000C840614908600020FFF7B6F901900198BE
:1079C00000284BD00198C0E6A06900282CD0584868
:1079D0000068FF210131084355490860FFF780F92D
:1079E000054606E0FFF77CF9401B022801D9032079
:1079F000ABE64F480068012149020840400A0028D0
:107A0000F0D04B484068072149038843216A084366
:107A100047494860084640680002000A217F09067D
:107A200008434349486019E041480068FF2101319B
:107A300088433F490860FFF753F9054606E0FFF722
:107A40004FF9401B022801D903207EE63848006820
:107A5000012149020840400A0028F0D1082120688D
:107A60000840082839D1606900281BD030484030D0
:107A70000069012108432E4940310861FFF730F9C0
:107A8000054606E0FFF72CF9401B022801D9032028
:107A90005BE6274840300069022108404008002882
:107AA000F0D01AE0224840300069400840002049E8
:107AB00040310861FFF714F9054606E0FFF710F9B9
:107AC000401B022801D903203FE6194840300069D5
:107AD0000221084040080028F0D104212068084015
:107AE000042879D1002000901148806B8906084055
:107AF000002806D10E48806B08430D498863012099
:107B000000900E480068FF210131084000281ED176
:107B10000A480068084309490860FFF7E1F805468C
:107B20000EE0FFF7DDF8401B642809D903200CE6BE
:107B300000100240BEB90008500100200070004053
:107B400085480068FF21013108400028E9D000BFC6
:107B5000FF210131A068884205D1804800690843AF
:107B60007E49086130E0A06800280DD17B4800699B
:107B7000FF210131884379490861084600690915E8
:107B80008843764908611FE005210902A068884200
:107B90000DD1724800690121890208436F490861CB
:107BA00008460069891508436C4908610CE06B4878
:107BB0000069FF210131884368490861084600696E
:107BC000091588436549086100BFA068002815D0E1
:107BD000FFF786F8054608E031E0FFF781F8401B23
:107BE0005F49884201D90320AFE55C480069012163
:107BF00049020840400A0028EFD013E0FFF770F870
:107C0000054607E0FFF76CF8401B5549884201D94B
:107C100003209AE551480069012149020840400AC1
:107C20000028EFD10098012808D14C484038806BDB
:107C300001210907884349494039886300BF606AC8
:107C400000284CD00C2E69D0606A022848D14348E5
:107C500040380068012109068843404940390860DE
:107C6000FFF73EF8054606E0FFF73AF8401B02280A
:107C700001D9032069E539484038006801214906E7
:107C80000840400E0028EFD1E16AA06A0843216B4A
:107C9000084332494039C968FD2212049143084320
:107CA0002E494039C860084600680121090608438A
:107CB0002A4940390860FFF713F8054606E0FFF748
:107CC0000FF8401B022801D903203EE52348403825
:107CD0000068012149060840400E0028EFD038E036
:107CE0001E48403800680121090688431B49403975
:107CF0000860FEF7F5FF054606E0FEF7F1FF401BC2
:107D0000022801D9032020E51448403800680121E9
:107D100049060840400E0028EFD11AE0606A0128A9
:107D200000D112E50D484038C768012000043840F2
:107D3000A16A88420BD10F2080043840E16A884252
:107D400005D1032080053840216B884201D00120F5
:107D5000FBE40020F9E40000007000404010024005
:107D60008813000010B50446002C01D1012010BD7D
:107D7000606A002800D100BF0021A1625120005D8F
:107D8000002804D150200155204600F035F802218A
:107D9000512001552068006840218843216808600F
:107DA000A16860680843E168084321690843616984
:107DB000084301225202A16911400843E1690843C6
:107DC000216A0843A16A084321680860A069000C81
:107DD00004210840616A0843216848602068C0693E
:107DE000910088432168C86100206065012151200D
:107DF00001550020BBE7000010B586B004461421F1
:107E000001A8FDF7E8F914492068884222D11348F7
:107E1000406B891408431149486300BF0846C06A93
:107E2000012108430D49C8620846C06AC007C00F57
:107E3000009000BF00BFE0200190022002900020CF
:107E40000390032004900020059001A9052000075D
:107E5000FEF740FE06B010BD0030014000100240A9
:107E6000FFB583B0044616461D4600200290E06828
:107E7000002804D1E068002802D1012E00D900BFFB
:107E8000FF210531606888420ED1A06800280BD11F
:107E900004215120015533460095049A114620468D
:107EA00000F088F907B0F0BD00BF5020005D012848
:107EB00001D10220F6E701215020015500BFFEF755
:107EC0000FFF07465120005D012802D002200290DA
:107ED00082E00498002801D0002E02D101200290F7
:107EE0007AE0042151200155002060650498A063C8
:107EF000A687E68700202063A086E0862064606471
:107F00004903A068884205D1206800684910884369
:107F1000216808602068006840210840402804D09B
:107F200020680068084321680860E068002822D1C2
:107F30001DE020688068C007C00F00280AD02068B4
:107F4000007BA16B0870A06B401CA063E08F401EFB
:107F5000E0870CE0FEF7C4FEC01BA84202D3681CF9
:107F6000002801D1002D02D10320029034E0E08FDF
:107F70000028DED121E01DE020688068C007C00F26
:107F800000280AD02068C068A16B0880A06B801C04
:107F9000A063E08F401EE0870CE0FEF7A1FEC01B4F
:107FA000A84202D3681C002801D1002D02D1032071
:107FB000029011E0E08F0028DED13A4629462046A3
:107FC00001F0D2FA002801D020206065606D002801
:107FD00001D00120029000BF01215120015500BFB6
:107FE00000215020015500BF02985BE7FFB583B028
:107FF000044616461D4600200290E068002804D181
:10800000E068002802D1012E00D900BF00BF502037
:10801000005D012802D1022007B0F0BD01215020EF
:10802000015500BFFEF75CFE074601965120005D3A
:10803000012802D002200290B2E00498002801D06A
:10804000002E02D101200290AAE003215120015507
:108050000020606504982063A686E6860020A06361
:10806000A087E087606420640121C903A06888427A
:1080700005D120680068491008432168086020681D
:10808000006840210840402804D020680068084368
:10809000216808600121C902E068884232D1606825
:1080A000002802D00198012809D1206B008821689E
:1080B000C860206B801C2063E08E401EE0861DE0BF
:1080C000206880680221084002280AD1206B0088BD
:1080D0002168C860206B801C2063E08E401EE08613
:1080E0000CE0FEF7FDFDC01BA84202D3681C00286F
:1080F00001D1002D02D10320029051E0E08E002832
:10810000DED131E06068002802D00198012809D151
:10811000206B007821680873206B401C2063E08E80
:10812000401EE0861DE02068806802210840022889
:108130000AD1206B007821680873206B401C2063F3
:10814000E08E401EE0860CE0FEF7CAFDC01BA84290
:1081500002D3681C002801D1002D02D10320029017
:108160001EE0E08E0028DED13A462946204601F086
:108170004CFA002801D020206065A068002809D1B1
:1081800000BF00902068C068009020688068009060
:1081900000BF00BF606D002801D00120029000BF29
:1081A00001215120015500BF00215020015500BF81
:1081B000029831E7FFB587B004461D46109E0120A6
:1081C000039000200290E068002804D1E0680028B5
:1081D00002D1012D00D900BF00BF5020005D012851
:1081E00002D102200BB0F0BD01215020015500BF8B
:1081F000FEF776FD07465120005D0490606805900B
:108200000695049801280DD0FF2105310598884274
:1082100005D1A068002802D10498042802D00220C9
:108220000290E9E00898002804D00998002801D0BD
:10823000002D02D101200290DEE05120005D0428D3
:1082400002D0052151200155002060650998A063E6
:10825000E587A58708982063E586A5860020206429
:1082600060642068006840210840402804D02068ED
:1082700000680843216808600121C902E06888425B
:108280004FD16068002802D00698012809D1206BE0
:1082900000882168C860206B801C2063E08E401E2F
:1082A000E08637E02068806802210840022811D16A
:1082B000E08E00280ED0039801280BD1206B008897
:1082C0002168C860206B801C2063E08E401EE08621
:1082D0000020039020688068C007C00F00280ED0DF
:1082E000E08F00280BD02068C068A16B0880A06BCD
:1082F000801CA063E08F401EE08701200390FEF702
:10830000EFFCC01BB04205D3701C002802D0032034
:10831000029071E0E08E0028C4D1E08F0028C1D126
:1083200050E06068002802D00698012809D1206B2F
:10833000007821680873206B401C2063E08E401E8B
:10834000E08639E02068806802210840022811D1C7
:10835000E08E00280ED0039801280BD1206B007806
:1083600021680873206B401C2063E08E401EE0866D
:108370000020039020688068C007C00F00280ED03E
:10838000E08F00280BD02068C068A16B0870A06B3C
:10839000401CA063E08F401EE08701200390FEF7A1
:1083A0009FFCC01BB04202D3701C002801D1002EDC
:1083B00002D1032002901FE0E08E0028C2D1E08F9E
:1083C0000028BFD13A463146204601F01EF9002868
:1083D00004D001200290202060650DE0A0680028F4
:1083E00009D100BF01902068C068019020688068B2
:1083F000019000BF00BF00BF01215120015500BF07
:1084000000215020015500BF0298EBE670B50446EC
:108410002546681E0949884201D901200CE0681EE2
:10842000074948610321081F00F048FF0020044964
:10843000886107200861002070BD0000FFFFFF0079
:1084400000E000E070477047FEB504462068C5694B
:1084500020680668206887682807000F0190019847
:1084600000280ED12020284000280AD020203040AB
:10847000002806D0206E002802D02046216E8847B2
:10848000FEBD019800287DD0F807C00F002804D158
:10849000FF20213030400028F5D0E807C00F002829
:1084A0000BD0FF2001303040002806D00120216889
:1084B0000862E06F01210843E0670220284000289D
:1084C0000AD0F807C00F002806D0022021680862F1
:1084D000E06F04210843E0670420284000280AD008
:1084E000F807C00F002806D0042021680862E06F5A
:1084F00002210843E0670820284000280ED02020F1
:108500003040002803D1F807C00F002806D008200B
:1085100021680862E06F08210843E067E06F0028E7
:1085200046D020202840002809D0202030400028B4
:1085300005D0206E002802D02046216E8847E06FCB
:1085400000902068806840210840402804D008211D
:1085500000980840002826D0204601F0FCFD206845
:10856000806840210840402819D1206880688843ED
:1085700021688860E06E00280DD02548E16E886390
:10858000E06E00E015E0FEF77BF8002810D0E06E0A
:10859000816B88470CE02046FFF755FF08E0204636
:1085A000FFF751FF04E02046FFF74DFF0020E06792
:1085B00066E701200005284000280CD00120800536
:1085C0003840002807D001200005216808622046B5
:1085D000FFF738FF54E78020284000280AD0802089
:1085E0003040002806D0606E002802D02046616E20
:1085F000884745E740202840002807D040203040E9
:10860000002803D0204601F0B8FD39E700BF37E766
:1086100095A0000810B50446002C01D1012010BD22
:10862000A069002800D000E000BF606F002805D1DD
:10863000002170200155204600F02CF824206067AE
:10864000206800684008400021680860204601F06A
:10865000FBFD012800D1E2E7606A002802D0204635
:1086600001F08AFB206840680921C902884321681B
:108670004860206880682A218843216888602068D3
:1086800000680121084321680860204601F0ECFBE6
:10869000C5E7000010B586B00446142101A8FCF718
:1086A0009AFD36492068884266D13548406B0121E1
:1086B000890308433249486300BF0846C06A012164
:1086C00008432F49C8620846C06AC007C00F00901F
:1086D00000BF00BF03204002019002200290002052
:1086E0000390032004900420059001A905200007B1
:1086F000FEF7F0F923482449086003204860002170
:1087000021488160C1608021016100214161816156
:108710002021C16100210162FEF764F8002801D028
:10872000FDF7C2FA00BF1848E066846200BF154832
:1087300014381649086003204860102113488160EE
:108740000021C16080210161002141618161C1611D
:108750000162FEF747F8002801D0FDF7A5FA00BF37
:108760000A48A066846200BF002201211B20FEF798
:10877000DFFC1B20FEF7D0FC06B010BD0038014026
:108780000010024030000240901A0020D81A002049
:1087900070B504460D461646A06F202863D1002D03
:1087A00001D0002E01D1012070BD01210903A06874
:1087B000884208D12069002805D1E807C00F0028A9
:1087C00001D00120F0E700BF7020005D012801D139
:1087D0000220E9E701217020015500BF656558209E
:1087E00006530020E0672220A067E06E002820D01A
:1087F0001E48E16EC8621E48E16E08631D48E16EC6
:1088000048630020E16E88632368194624313346AB
:10881000626DE06EFEF73AF800280AD01020E0679B
:1088200000BF00217020015500BF2020606701209B
:10883000BAE700BF00217020015500BF2068006822
:10884000FF21013108432168086020688068012108
:1088500008432168886020688068402108432168B7
:1088600088600020A0E702209EE70000FFA000082B
:1088700049A10008ADA0000870477047FFB583B05C
:1088800004460D461746606F202875D1002D01D093
:10889000002F02D1012007B0F0BD01210903A0681B
:1088A000884208D12069002805D1E807C00F0028B8
:1088B00001D00120EFE700BF7020005D012801D149
:1088C0000220E8E701217020015500BF0020E06789
:1088D00021206067FEF704FA0190502007535220D0
:1088E000075301210903A068884205D120690028A7
:1088F00002D10026029502E02E460020029021E0DF
:1089000006980090002280212046019B01F08AFEFB
:10891000002801D00320BEE7002E09D1029800886C
:10892000C005C00D216888620298801C029003E097
:10893000307821688862761C5220005B401E81B22C
:10894000522001535220005B0028D9D10698009094
:10895000002240212046019B01F064FE002801D046
:10896000032098E72020606700BF00217020015598
:1089700000BF00208FE7FFE702208CE7704700BFB1
:10898000FEE710B50022042105200007FEF7A1F93B
:108990000022082105200007FEF79BF90A2002F0BB
:1089A000C9F90122042105200007FEF792F90A20E7
:1089B00002F0C0F90022042105200007FEF789F922
:1089C00010BD10B50022042105200007FEF781F933
:1089D0000122082105200007FEF77BF90A2002F09A
:1089E000A9F90122042105200007FEF772F90A20E7
:1089F00002F0A0F90022042105200007FEF769F922
:108A000010BD70B50546002400261EE0002204219A
:108A100005200007FEF75DF90A2002F08BF901221C
:108A2000042105200007FEF754F96006040E082112
:108A300005200007FEF744F9002801D0601CC4B2ED
:108A4000052002F077F9701CC6B2082EDEDB002D7F
:108A500002D1FFF7B6FF01E0FFF793FF204670BD9C
:108A600070B504460022042105200007FEF731F905
:108A700000252AE080202040C011002806D00122D5
:108A8000082105200007FEF724F905E0002208214F
:108A900005200007FEF71DF96006040E0A2002F00B
:108AA00049F90122042105200007FEF712F90A20E6
:108AB00002F040F90022042105200007FEF709F921
:108AC0000A2002F037F9681CC5B2082DD2DB70BD50
:108AD00010B50122082105200007FEF7FAF801224F
:108AE000042105200007FEF7F4F8002208210520E4
:108AF0000007FEF7EEF80A2002F01CF9002204211C
:108B000005200007FEF7E5F810BD10B5002204218E
:108B100005200007FEF7DDF80022082105200007E8
:108B2000FEF7D7F80A2002F005F9012204210520FA
:108B30000007FEF7CEF80122082105200007FEF706
:108B4000C8F80A2002F0F6F810BD10B50024012282
:108B5000082105200007FEF7BCF8062002F0EAF81D
:108B60000122042105200007FEF7B3F8062002F0D9
:108B7000E1F807E0601CC4B2FA2C03DDFFF7C5FF83
:108B8000012010BD082105200007FEF799F80028F4
:108B9000F0D10022042105200007FEF79AF80020FA
:108BA000EFE7000038B500203D49087001F094F966
:108BB00001F0E6F93B480068C06908210840002838
:108BC00002D039483949C86080213948FEF778F821
:108BD00000280BD1012251033548FEF77AF8002214
:108BE000012109033248FEF774F811E00022012147
:108BF00049032F48FEF76DF80121C9022C48FEF702
:108C00005FF8002804D0012211032948FEF761F81B
:108C10002848808C012820D100242748009072B673
:108C200080212648FDF75CF80446002C05D002227E
:108C300069462248FDF746F9044662B620A001F0D5
:108C400027FE00211B48818402F034FE642002F0DC
:108C500067F815481549C86000BF1648408C0128C0
:108C60000ED1002113484184002012494039088068
:108C700002F020FE642002F053F80B480B49C86054
:108C80000C48008C01280AD100210A48018402F016
:108C900011FE642002F044F803480449C86038BD5E
:108CA000E7000020101A00200400FA0500ED00E0A3
:108CB00000040050C40D0020AAAA0000384A000891
:108CC000BDF8C8EBC9FDBCB6C4A3CABD0D0A0000FF
:108CD00008B53721202000F073F80321212000F08F
:108CE0006FF84021222000F06BF80821232000F0CB
:108CF00067F8AA21302000F063F80A48008FC1B25B
:108D0000322000F05DF80221332000F059F85F2195
:108D1000202000F055F8684600F006F80A2002F01E
:108D200009F808BD840D002010B5044621460F2027
:108D300000F023F8002800D110BD0120FCE770B539
:108D400004460025FFF7C4FE3220FFF789FEFFF737
:108D5000FCFEE0B2FFF784FEFFF7F7FEFFF7B8FE78
:108D60003320FFF77DFEFFF7F0FE0020FFF749FEFE
:108D70000546FFF7CAFE284670BD70B505460C468D
:108D80002846FFF7DCFF2070012070BD70B5044657
:108D90000D46FFF79DFE3220FFF762FEFFF7D5FE7E
:108DA000E0B2FFF75DFEFFF7D0FE2846FFF758FE62
:108DB000FFF7CBFEFFF7A9FE0A2001F0BBFF70BD55
:108DC00070B504460D4629462046FFF7DFFF012017
:108DD00070BD000010B50248FEF735F810BD000068
:108DE00088190020F0B585B004460020039072B6C3
:108DF0004F4920684018002806D14E48C06803211A
:108E000089040840039000E000BF00BF206880682C
:108E100002902068C06801902068456920688669D2
:108E200043492068401800280DD142484038806AE4
:108E3000490508433F49403988620846806A400036
:108E40004008886200E000BF00BF002D01D1002E65
:108E50005FD0374920684018002807D13548C068DE
:108E60000321890488433349C86000E000BF00BF84
:108E7000002D1DD020680069012108432168086188
:108E800020684561FDF72CFF074600BFFDF728FF6E
:108E9000C01B00902068006808210840082804D002
:108EA0007D21C90000988842F0D9082021684860D7
:108EB000002E1DD020680069012108432168086147
:108EC00020688661FDF70CFF074600BFFDF708FF2D
:108ED000C01B00902068006810210840102804D0B2
:108EE0007D21C90000988842F0D91020216848608F
:108EF0000F4920684018002809D10E48C068032196
:108F000089048843039908430A49C86000E000BF08
:108F100000BF20680069400840002168086102988D
:108F20002168886001982168C86062B605B0F0BD0C
:108F30000084FFBF401002401CB50020009001904B
:108F40001E481F49086000211D48C1630120800799
:108F50001B49486000211A48816007218163012173
:108F600001610021C160001D01774177001F81620E
:108F7000FF21C231416200212430017204212438D2
:108F800041610021016381614163C161FDF778F9AD
:108F9000002801D0FCF788FE0A4800908013019059
:108FA00069460748FDF7E0F8002801D0FCF77CFE91
:108FB00000210348FDF76AF81CBD000000240140B1
:108FC0002C1900200200000408B500BF0A48006BFD
:108FD00001210843084908630846006BC007C00F19
:108FE000009000BF00BF002201210A20FEF7A0F878
:108FF0000A20FEF791F808BD0010024000B587B0C6
:10900000142102A8FCF7E7F800BF6548C06A0421F4
:1090100008436349C8620846C06A042108400190B9
:1090200000BF00BF00BF5E48C06A802108435C49A2
:10903000C8620846C06A80210840019000BF00BF96
:1090400000BF5748C06A012108435549C862084615
:10905000C06AC007C00F019000BF00BF00BF084634
:10906000C06A022108434E49C8620846C06A02210C
:109070000840019000BF00BF01221C21052000070D
:10908000FDF727FE012291024648FDF722FE00224D
:1090900045494448FDF71DFE0022912109020520A3
:1090A0000007FDF716FE01200290404803900020C3
:1090B000049002A905200007FDF70CFD0220029094
:1090C000032003900020049002A905200007FDF76B
:1090D00001FD0C2002901120039000200490032039
:1090E000059002A905200007FDF7F4FC102002906E
:1090F00001200390002004900220059002A9052081
:109100000007FDF7E7FC01200290112003900020EA
:109110000490059002A92348FDF7DCFC0220029090
:10912000234803900120049002A91E48FDF7D2FCB9
:10913000204802900120039000200490059002A98D
:109140001848FDF7C7FC0120C002029000200390E0
:109150000220049002A91348FDF7BCFC91200002F4
:1091600002900120039000200490059002A90520A0
:109170000007FDF7AFFC8020029000200390012043
:10918000049002A90748FDF7A5FC00220121052053
:10919000FDF7CEFF0520FDF7BFFF07B000BD0000C3
:1091A00000100240000400500930000000001110BF
:1091B000000021100834000010B50F480F49086066
:1091C0000020486000210D4881600D494161002167
:1091D000016241628162FDF7C1FE002801D0FCF707
:1091E00063FD084A511C0548FDF748FF002801D0DF
:1091F000FCF75AFD10BD0000007C004088190020DB
:10920000FFFF0000FF7F000010B512481249086000
:10921000FF200530486000210F488160C160016176
:1092200041610121490281610021C1610162416204
:1092300081620721C162FEF795FD002801D0FCF78D
:1092400033FD054800680068402108430249096869
:10925000086010BD00300140B819002010B5134857
:1092600013490860E12040024860002110488160F5
:10927000C16001610C21416100218161C161016214
:1092800000200B4948620846FFF7C4F9002801D0C6
:10929000FCF70AFDC82207490548FFF779FA0028BC
:1092A00001D0FCF701FD01F0FFF910BD00380140CD
:1092B000101A0020BC0C00207047000010B50028D8
:1092C00019DA1A4A03071B0F083B9B089B00D25868
:1092D0008307DC0EFF23A3409A438B071B0E8407F2
:1092E000E40EA3401A43114B0407240F083CA408C2
:1092F000A4001A5118E00E4A03231B02D218830857
:109300009B00D2588307DC0EFF23A3409A438B07B0
:109310001B0E8407E40EA3401A43054B03242402CA
:109320001B198408A4001A5110BD00001CED00E0B8
:1093300000E100E070470000F0B585B04E484F49AD
:10934000086002F057FAFF2009304D4948800A2092
:1093500048870846C08E4B4908704948C08F4A4923
:1093600008704748808F494908704548807A4849C5
:109370000870434880884749086041490889FCF7DC
:10938000CFF906460022444BFCF7C4F804460022FD
:10939000424BFCF727F90191009001F05DFC03912D
:1093A0000290FCF7DFF93E4908803549C8883C49FE
:1093B0000988FBF7B3FE3B49088031498888394961
:1093C0000988FBF7ABFE36480088414388B236492E
:1093D0000880084600880A30FCF77CF9334902907F
:1093E000FBF76AFF0390FCF7DBF90646304A314B86
:1093F000FCF7F8F80446FCF7B5F92F490880084651
:1094000000882E4908801E49C888FCF76EF9274954
:109410000290FBF751FF0390FCF7C2F90446244A7F
:10942000244BFCF7DFF80646FCF79CF9244908803A
:109430001348C1887D20C000FBF770FE21490880D9
:109440001D48028820492148FDF718FE002801D058
:10945000FCF72AFC0F4801681DA001F019FA084822
:10946000C1881FA001F014FA0548018921A001F06C
:109470000FFA05B0F0BD0000B5A6000848000020B6
:10948000840D002001000020380100203901002057
:10949000270100201C0100200000104000000840AF
:1094A0002C0100202E0100202801002000007A4419
:1094B000F853E3A59B843E40340100203001002096
:1094C0003201002036010020478100008819002069
:1094D000B1EAC7A949443A202564202E0D0A0000AC
:1094E000CDA8D1B6BCE4B8F43A202564206D732E23
:1094F0000D0A0000B5A5B4CECDA8D1B6BBF9D5BE36
:10950000CAFDC1BF3A202564B8F62E0D0A0000003E
:1095100000B585B014216846FBF75DFE00220121ED
:10952000C9031048FDF7D5FB0120C00300900120BE
:10953000019000200290039069460A48FDF7CAFA9C
:109540000120C003009003200190002002900390AE
:1095500069460448FDF7BEFA022001F0E1FB05B0C0
:1095600000BD000000040050F8B504460E46154644
:10957000FF210531606888420ED10121C903A0682E
:10958000884203D04911A068884205D1206800684C
:109590004021884321680860FF21053160688842C6
:1095A00022D101218902A06888420ED033460022D0
:1095B00080212046009500F055F8002823D0606DEA
:1095C0002021084360650320F8BD334600220121B5
:1095D0002046009500F046F8002814D0606D202148
:1095E000084360650320EFE733460022012120464F
:1095F000009500F037F8002805D0606D2021084361
:1096000060650320E0E70020DEE7F8B504460E467B
:109610001546FF210531606888420ED1334600228D
:1096200080212046009500F01DF8002818D0606DBC
:109630002021084360650320F8BD5120005D052806
:109640000ED13346002201212046009500F00AF891
:10965000002805D0606D2021084360650320EBE7FA
:109660000020E9E7F8B504460E4617461D4641E0DE
:10967000681C00283ED0FDF733FB0699401AA8422B
:1096800001D2002D36D120684068E021884321684E
:109690004860FF210531606888420ED10121C9036D
:1096A000A068884203D04911A068884205D120688B
:1096B0000068402188432168086001214903A06AAD
:1096C00088420DD100BF2068006888432168086087
:1096D000206800680121490308432168086000BF31
:1096E00001215120015500BF00215020015500BF2C
:1096F0000320F8BD206880683040B04201D10120CD
:1097000000E00020B842B3D10020F2E7704700002B
:1097100038B504460D460020009055201B490870BE
:10972000AA20487003208870601DC870032008714B
:109730000846457184716800154A8118224613480D
:10974000C01DFBF72FFD002008E0811C0F4A525C72
:109750006946098851188AB20092401C611D8842EE
:10976000F3DB0A48801CFCF7EDF90090E01D074987
:10977000411868460078087068464078487021466D
:109780000931024800F012FD38BD0000C718002062
:10979000840D002001460020054A126890B2054A57
:1097A000104002460A431046014A1060704700000C
:1097B00000300140C7FF000010B5FDF797FA10BD5B
:1097C00000B599B034210CA8FBF705FD142107A8BA
:1097D000FBF701FD1C216846FBF7FDFC24480068EF
:1097E0000321C90288430121C902401820490860A9
:1097F000FDF7B0FC1F4800690321C90288431D49D9
:10980000086106200C9088150E9001200F90102002
:1098100010900220159000211691410417914105E6
:1098200018910CA8FDF78CFF002801D0FCF73CFA3A
:109830000F20079003200890002009900A900B90B9
:10984000012107A8FDF7E6FD002801D0FCF72CFA5E
:10985000812000900020029003208004069068463A
:10986000FDF7C2FC002801D0FCF71EFA19B000BDBC
:10987000007000404010024015480068FF2101318F
:109880000843134908600846C06812490840104957
:10989000C86008460068104908400D49086008463D
:1098A00080684008400088600846006801218904FB
:1098B0008843074908600846C068FD2109048843B9
:1098C0000349C86000200861044805498860704762
:1098D000001002400C40FF88F6FFF6FE0050000822
:1098E00000ED00E0F0B58DB000200A9001F0E4FC3E
:1098F0000B9002E001F0E0FC0B90F4490B988842D9
:10990000F8D10020F2490880962001F030FD4B206C
:10991000C00001F049FD0020EE490870EE480078D3
:10992000EE49C873EE4801780068401CEC4A1060AC
:10993000C8B2EA4948740025BFE1E84885730022AF
:109940000146142001F016FE0021142001F026FE2D
:10995000022001F067FDE3490870E348076805E06D
:1099600000210F2001F08EFCE049086000210F204B
:1099700001F088FCDD490860DD4908400028EFD08F
:10998000DA48006801218903084000287DD081223F
:10999000D20100210F2001F0A6FD0021102001F0CE
:1099A00071FC4006400ED34908600846008881B229
:1099B0000022D14801F0B6FCCF480078CF490978A1
:1099C00088427DD1CC48407A0228FAD10422CC4981
:1099D000C948401DFBF70AFC0028F2D101F03BFE0C
:1099E000C84A03C201F020FEC74A03C20A980028F1
:1099F0002AD1C648C089002826D001200A90C4492F
:109A0000BD48C0890880C348BB49098A01800088D5
:109A1000FF30C330BF49088008460088BE498842ED
:109A200012DDBC480088401ABA490880B84800884E
:109A3000401CB749088008460088B7490B31884266
:109A400002DB0020B2490880B449AB4842890A8051
:109A5000808948800422A849491CB148FBF7A2FB31
:109A6000A548418A08916846008C042813DDA74860
:109A7000C0886946098C88420DD06846008CA3498D
:109A8000C88001F017FF642000E00CE101F048F904
:109A9000A448A549C8609C4803684068A34A0021BF
:109AA0009A1848410106140A0C43204601F057FC5D
:109AB0006108490000200A0E000210430B0200E07A
:109AC000EDE0002211469A18484199490A60486021
:109AD0008C480CC89248093001F08CFD8A480CC8AB
:109AE0008F480D3001F086FD91480CC88C4811302C
:109AF00001F080FD00228A49491E182001F03AFD3C
:109B00000021182001F04AFD012001F08BFC75496D
:109B100008707F4800887D21C90048437D49098835
:109B20004018844908608448FDF7A4FA86B2774A51
:109B3000D2887D23DB005A4311467E4A12687F4B50
:109B4000D01AFBF7EBFA7E4800887D22D200504302
:109B50006E4AD2887D23DB005A438018401A794927
:109B6000401A7949086073490968784A881A0028B8
:109B700001DB014600E041427D22D200914205DA3C
:109B8000714800686D4940186F4908606E48006868
:109B90007D210901884208DA5C48C08849104843A1
:109BA0006949096840186849086067480068FBF718
:109BB000A3FD674A674B01910090FBF713FD0591E8
:109BC00004903046FBF7ACFD03910290059B049A8C
:109BD000FBF7EEFB07910690FBF7C4FD5E4908809A
:109BE000084600885D49884204DD5B480088401AC9
:109BF00059490880584800884F49096848613548E4
:109C00000078401C334908703B48427808A90A7123
:109C1000807848713D48C08B00282AD101205049E6
:109C200088701120C8702E480078087108463449A1
:109C30000A784271497881712F494A78C2718978CE
:109C40000172042235490930FBF7ACFA4548007827
:109C50004349487344480078887311214048801C68
:109C6000FBF770FF414908803D480A78C274497883
:109C700001751C480078002808D100BF00210F2082
:109C800001F000FB802108400028F7D0802200214D
:109C90000F2001F028FC0020354908700BE001205E
:109CA0003349087007E0334A00210F2001F01BFC04
:109CB00001202F490870681CC5B214480089A842C9
:109CC00000DD3AE601F0CCF90DB0F0BD3001CADE9E
:109CD000E8000020EB000020420100208415002055
:109CE0006C000020EA000020FC000020740000202E
:109CF00000D0272404010020D415002027010020D3
:109D00001C0100207800002080000020840D00202D
:109D100024010020F8000020E7030000F0000020EC
:109D2000A71500200400FA0500ED00E00000520332
:109D30008800002000010020881900201027000062
:109D4000280100201E1400000C010020B0E20D00CC
:109D5000F853E3A59B843E4030010020478100007A
:109D60004A180020E4000020E5000020F400002054
:109D7000B800002000902724818CC907C90F002952
:109D800008D001684968012252049143826A114354
:109D9000026851600222416A1140022907D101681C
:109DA0004968D2039143C26A114302685160042298
:109DB000416A1140042907D101684968120491439E
:109DC000026B1143026851600822416A1140082960
:109DD00007D10168496812039143426B114302683D
:109DE00051601022416A1140102907D10168896829
:109DF00012029143826B1143026891602022416AF2
:109E00001140202907D10168896812029143C26B71
:109E10001143026891604022416A1140402915D1E6
:109E20000168496892039143026C114302685160D2
:109E300001221205016C914208D101684968032290
:109E400052059143426C1143026851608022416A7D
:109E50001140802907D10168496812039143826C3F
:109E6000114302685160704738B504460020E0672E
:109E7000FCF736FF054620680068082108400828DE
:109E80000BD114482B46002289040090204600F094
:109E9000C9FB002801D0032038BD206800680421D8
:109EA000084004280BD10B482B46002209050090DE
:109EB000204600F0B7FB002801D00320ECE720206B
:109EC0006067A06700BF00217020015500BF00201F
:109ED000E2E70000FFFFFF0170B50025C82420481D
:109EE0000078002800D070BD1E480078002800D0FF
:109EF000F9E701201B4908701B48406B002801D17D
:109F00000870F0E71848406BC8210D1A1CE017498B
:109F1000174A1268885C17490968884716480088FC
:109F20003C2148431549088011480068401C1049ED
:109F3000086008460068C82801DB002008600A485D
:109F4000406BC8210D1A641E09480068A84201D060
:109F5000002CDCDC00200349087000BFC3E70000D0
:109F6000420000204400002000000240BC0C002001
:109F70003800002048000020360100204001002069
:109F800010B53A480078002803D1394800780028F5
:109F900000D010BD0120364908703648C0698021C4
:109FA0000840002802D132490870F2E73249002007
:109FB0000856324900228A56904215D12D48C06970
:109FC0004021084000280BD02D480078002807D0F9
:109FD00000202B4908702B480088401C2949088024
:109FE000002023490870D4E725480078002805D1CF
:109FF0000120234908700A2000F09CFE1F49002020
:10A000000856CC21484320494018001D1F490968C3
:10A01000405C184988621D480068401C1B49086064
:10A02000164900200856CC214843174908581749BB
:10A030000968884214DC0020144908600F48007841
:10A04000401C40B20D490870084600780E2801D126
:10A05000002008700E480078401C40B20C4908707F
:10A0600000200349087000BF93E700004200002071
:10A07000430000200038014035000020340000205B
:10A0800045000020520000209401002058000020CC
:10A090003600002070B50546AC6A00215A200153F5
:10A0A000522001532046FEF7CEF970BDF8B50546A3
:10A0B000AC6A666FA76F206880688021084080289E
:10A0C00007D1212E05D1002152200153204600F056
:10A0D00064F82068806840210840402807D1222F7A
:10A0E00005D100215A200153204600F034F8E06FDA
:10A0F00010210843E0672046FEF7A5F9F8BD70B5CA
:10A100000546AC6A2868006820210840002817D15D
:10A1100000215A20015320680068FF210131884343
:10A1200021680860206880684008400021688860D5
:10A130002068806840218843216888602020A067CB
:10A140002046FEF799FB70BD70B50446A56A284607
:10A15000FEF793FB70BD01680968FF22213291432D
:10A1600002681160016889684908490002689160C5
:10A170002021816700210166704710B504462068E0
:10A180000068402188432168086020206067002023
:10A1900060662046FEF7F2FB10BD01680968C02228
:10A1A00091430268116020214167704770B50546F0
:10A1B0000C4620480078002803D11F48007800286A
:10A1C00000D070BD01201B490870C82C04DC1B485E
:10A1D00000214156002903DC002016490870F0E7F1
:10A1E000174900200856CC21484316490C50144A00
:10A1F00000215156CC225143124A8918081D22468B
:10A200002946FAF7CFFF0E480078401C40B20C49AF
:10A210000870084600780E2801D100200870074811
:10A220000078401E40B205490870002001490870BE
:10A2300000BFC6E742000020430000203600002097
:10A240003500002094010020F0B587B004461020AE
:10A2500004900025002003900026E74920688842EA
:10A2600000D100E000BF2169A0680843616908438C
:10A27000E1690843074620680068E0490840384320
:10A280002168086020684068032109038843E16869
:10A29000084321684860A769D7492068884201D0EF
:10A2A000206A0743206880680B21090288433843ED
:10A2B0002168886000BFD249206888421CD1D148FB
:10A2C000C0688007800F002806D001280AD0022825
:10A2D00005D003280CD108E0012004900BE00220F7
:10A2E000049008E00420049005E00820049002E0B7
:10A2F0001020049000BF46E0C349206888421CD16A
:10A30000C048C0680C210840002806D004280AD0A4
:10A31000082805D00C280CD108E0002004900BE0A0
:10A320000220049008E00420049005E00820049036
:10A3300002E01020049000BF25E0AF492068884269
:10A340001FD1B048C068032189020840002808D006
:10A3500001218902401A0AD0401A05D0401A0CD1B6
:10A3600008E0002004900BE00220049008E00420A4
:10A37000049005E00820049002E01020049000BF43
:10A3800001E01020049000BF9B492068884256D10C
:10A39000049804281AD004DC002807D002281CD115
:10A3A00008E0082816D0102817D117E0FDF73CF96F
:10A3B000064616E09348403800681021084000091E
:10A3C000002801D0914E00E0914E0AE0FDF750F9CF
:10A3D000064606E00126F60303E000BF01200390D5
:10A3E00000BF00BF002E0AD0606841004018B04294
:10A3F00003D860680003B04202D201200390F4E069
:10A40000606802903046FF21013100F068FA62680E
:10A41000520800238018594101910090029AFAF7DE
:10A4200091FE054603200002854205D37948854206
:10A4300002D82068C560D8E001200390D5E0012152
:10A44000C903E06988426FD1049804283CD006DC37
:10A45000002809D0012813D002284AD11CE008287E
:10A460003ED0102845D145E0FDF7DEF84000616898
:10A470004908401802906168FAF73AFE85B23CE05C
:10A48000FDF7E4F8400061684908401802906168EF
:10A49000FAF72EFE85B230E05A48403800681021A5
:10A4A00008400009002807D061684A085A4BD018B4
:10A4B000FAF71EFE85B206E061684A08574BD018CD
:10A4C000FAF716FE85B218E0FDF7D2F84000616891
:10A4D0004908401802906168FAF70AFE85B20CE05C
:10A4E00061684A0801231B04D018FAF701FE85B2FF
:10A4F00003E000BF0120039000BF00BF102D0FD369
:10A50000474885420CD846480F3828400590280710
:10A51000400F05990843059005982168C86064E0DC
:10A520000120039061E0FFE7049804283AD006DC9C
:10A53000002809D0012812D0022847D11AE00828A3
:10A540003BD0102842D142E0FDF76EF8616849081F
:10A55000401802906168FAF7CBFD85B23AE0FDF74A
:10A5600075F861684908401802906168FAF7C0FD03
:10A5700085B22FE0234840380068102108400009C8
:10A58000002807D061684A08204BD018FAF7B0FDC0
:10A5900085B206E061684A081D4BD018FAF7A8FD9D
:10A5A00085B217E0FDF764F8616849084018029029
:10A5B0006168FAF79DFD85B20CE061684A080123E5
:10A5C000DB03D018FAF794FD85B203E000BF012049
:10A5D000039000BF00BF102D05D31148854202D85B
:10A5E0002068C56001E001200390002020666066BD
:10A5F000039807B0F0BD000000480040F369FFEF8A
:10A6000000380140401002400044004000093D0075
:10A610000024F400FFFF0F0000127A000048E80158
:10A62000FFFF0000FFB581B004460D4617460A9EA5
:10A6300022E0701C00281FD0FCF752FB0499401A3E
:10A64000B04201D8002E17D120680068FF21A13147
:10A6500088432168086020688068400840002168BD
:10A66000886020206067A06700BF0021702001552E
:10A6700000BF032005B0F0BD2068C0692840A84293
:10A6800001D1012000E00020B842D2D00020F1E743
:10A6900010B510200349096808620248FDF7D4FE8E
:10A6A00010BD0000101A00200D20014908707047ED
:10A6B0003600002070B5044600256A480078082856
:10A6C00065D100BF002004E06749095C49198DB2DB
:10A6D000401C66490978491F8142F5DC64480078CE
:10A6E000281885B261480078281885B2614800783A
:10A6F000281885B260480078281885B25F4800782D
:10A70000281885B26019C007C00F002835D05848F6
:10A710000078012827D002282DD15949554A1278AE
:10A72000881855490A785049FAF73CFD01F0C2F8FB
:10A73000642000F0F5FA00BF00BF00BF00BF00BFFB
:10A74000BFF34F8F00BF00BF00BF4E484E49C860E7
:10A7500000BF00BF00BFBFF34F8F00BF00BF00BFEF
:10A7600000BF00BFFDE74348007841104248007831
:10A77000FEF7CEFF00E000BF00BF0020394908709F
:10A780003C490870394908704049087068E035480C
:10A790000078072812D134483C49097844543B4892
:10A7A0000078401C3949087030480078401F09780B
:10A7B000884255D108202B49087051E0294800787B
:10A7C000062805D12C48047007202649087047E068
:10A7D00024480078052805D1264804700620214920
:10A7E00008703DE01F480078042805D12048047017
:10A7F00005201C49087033E01A480078032808D166
:10A800001A48047000201B4908700420154908707C
:10A8100026E014480078002805D1552C03D10120EA
:10A82000104908701CE00F480078012805D1AA2CB7
:10A8300003D102200B49087012E00A480078022870
:10A8400007D1032C05D10320064908700B4804707A
:10A8500006E00020034908700649087003490870A3
:10A8600070BD0000120100206318002014010020B8
:10A8700017010020150100201301002016010020FF
:10A88000840D00200400FA0500ED00E0180100200E
:10A890000FB410B503A9044B044A029800F034F930
:10A8A00010BC08BC04B0184711B6000854010020C1
:10A8B0002021020C01D010211046020A01D01046BE
:10A8C0000839020901D01046091F820801D010463C
:10A8D000891E420801D0881E7047081A7047F8B5D3
:10A8E00082B28BB2040C0D0C104658430021264650
:10A8F0005E43370C36048019794116466E43370C97
:10A9000036048019794126466E438919F8BD30B462
:10A910007446641E2578641CAB4204D3635D5B00FF
:10A92000E31830BC18471D46F8E702E008C8121FBC
:10A9300008C1002AFAD170477047002001E001C128
:10A94000121F002AFBD1704708B5002100916B4609
:10A95000012202212C2000F0DBFD022100916B4638
:10A9600001222C2000F0D4FD08BD000038B50446BB
:10A970006D2000906B46012208492E2000F0C8FD92
:10A98000002C05D0064A07492E2000F09BFD04E06C
:10A99000054A04492E2000F095FD38BD0608000048
:10A9A00007060000061800000716000038B5044628
:10A9B0006B4602220021362000F084FC2300FFF7C2
:10A9C000A6FF0E11081A54545454233154543D44D4
:10A9D0004B540021684601704078FE2108406946CA
:10A9E000487043E069460878FC210840012108438B
:10A9F000694608703AE069460878FC21084002215F
:10AA000008436946087031E068460078B321084081
:10AA10004821014368460170407880210843694617
:10AA2000487023E068460178B32001406846017011
:10AA300040784106490E6846417017E069464878FB
:10AA4000022108436946487010E069464878FD21B4
:10AA500008406946487009E069460878CF210840F7
:10AA6000202108436946087000E000BF00BF6B4624
:10AA700001220021362000F04BFD00AB0133012202
:10AA80001146362000F044FD38BD08B50321684664
:10AA90004170012101706B4602220021362000F036
:10AAA00037FD0122D20306212D2000F00BFD0120ED
:10AAB00000F036F90120FFF779FF08BD38B50446EC
:10AAC0002004010E6846417004706B460222042186
:10AAD0002D2000F01DFD0321684601706B46012208
:10AAE00006212D2000F014FD0021684601706B4600
:10AAF000012206212D2000F00BFD0A212D2000F05F
:10AB0000C1FB0546284638BDFFB58DB0044600257B
:10AB100006E025280AD0109A0F999047641C6D1CF6
:10AB200020780028F5D1284611B0F0BD002701217A
:10AB3000484A009700E00743641C23780846203BFE
:10AB400098401042F7D120782E2817D104200743CF
:10AB50006078641C2A280CD10E98641C02C80091ED
:10AB60000E900BE000990A22514330394018641CC2
:10AB700000902078014630390929F3D9207800283F
:10AB8000D1D0642808D0692806D075281ED0109A24
:10AB90000F9990476D1C5BE00A200E99019001C946
:10ABA0000E91002802DA40422D2102E0390504D539
:10ABB0002B216A461172012103E0F90704D02021FC
:10ABC000F7E70BAE0B910DE00021FAE70A200E9992
:10ABD000019001C90E91F7E70199FAF789FA30312E
:10ABE000761E31700028F7D103A8801B2030019019
:10ABF000780701D5009801E0012000900199884272
:10AC000001DD401A00E000200027009006E002A8C5
:10AC1000109AC05D0F9990476D1C7F1C0B9887425E
:10AC2000F5DB04E0109A30200F9990476D1C0099D5
:10AC3000481E00900029F5DC05E03078109A761C5B
:10AC40000F9990476D1C0199481E01900029F4DC72
:10AC5000641C65E709280100F8B54A002B4B520D2A
:10AC6000D6182B4A0C460546142E2BDA002E12DA83
:10AC7000284BFAF79DFB00221346FAF7A5FD40D2B8
:10AC8000002C03DA0124E40700253AE0204628439B
:10AC900037D0214C14E0214F0B46F7403B402B436B
:10ACA00031D01C4BFAF784FB00221346FAF78CFDD7
:10ACB00027D2002C03DD01200005F0400419BC431D
:10ACC00000251EE0332E1EDC33460027143BFF43D5
:10ACD000DF40384217D00F4BFAF714FC002213461E
:10ACE000FAF772FD0DD2002C0ADD142E0CD03420A0
:10ACF000811B012088404019A84200D2641C0546EF
:10AD0000BD4321462846F8BD641CF9E701FCFFFF5E
:10AD10009C7500883CE4377E0000F03FFFFF0F0089
:10AD200070B504467D20C00060430546284600F00B
:10AD300001F870BD002100BF40E000BF00BF00BFB0
:10AD400000BF00BF00BF00BF00BF00BF00BF00BF0B
:10AD500000BF00BF00BF00BF00BF00BF00BF00BFFB
:10AD600000BF00BF00BF00BF00BF00BF00BF00BFEB
:10AD700000BF00BF00BF00BF00BF00BF00BF00BFDB
:10AD800000BF00BF00BF00BF00BF00BF00BF00BFCB
:10AD900000BF00BF00BF00BF00BF00BF00BF00BFBB
:10ADA00000BF00BF00BF00BF00BF00BF00BF00BFAB
:10ADB00000BF00BF00BF00BF00BF491C8142BCD321
:10ADC00070470000F0B585B0044600200490039061
:10ADD0002578607940008A49085A02906078401EC0
:10ADE0008849C6B20863042D01D0072D01D1012086
:10ADF00000E000200190207882490873E079002863
:10AE00000AD1084680690121890508437D49886186
:10AE10000298C010029006E07A48806901218905F5
:10AE2000884378498861207A764948730846806962
:10AE3000217A0904032212041140084371498861F0
:10AE4000084600218269042000F04DFB6E492E2047
:10AE5000029A00F037FB3046FFF788FD6B48405DF3
:10AE6000810040186A494318052207212B2000F071
:10AE70004FFB684901980B1801220B21282000F094
:10AE800047FB6248405D800063490A580C21282036
:10AE900000F029FBE079800060494018A179490061
:10AEA000425A0221272000F00DFB70005C490A5A2B
:10AEB0000421272000F006FBE079002805D1642258
:10AEC0000621272000F0FEFA1EE0A07804280DD10C
:10AED0001020009010220621272000F0F3FA6B4684
:10AEE00001222621272000F013FB0DE028200090EE
:10AEF00020220621272000F0E5FA6B4601222621B8
:10AF0000272000F005FB00BF300146494018E178DA
:10AF1000890042580821272000F0E5FAA17A627AD8
:10AF200008021043002803D13F496172090AA17247
:10AF3000A17A637A0802184302462021272000F0F4
:10AF4000C1FA3A480C210268232000F0CCFA7100C3
:10AF50003648001D425A0421232000F0B3FAA0799C
:10AF600000280BD0E079324943180122002121202A
:10AF700000F0CEFA03200490012003902807000F70
:10AF80002901F022114008436178890403229204C8
:10AF900011400843049909059200114008430399A0
:10AFA00049040122520411400843217989051F22D6
:10AFB0009205114008436179C906C90EC9060843C4
:10AFC00007463A4600211F2000F08DFAA0786178EC
:10AFD000084300040B49086108460069E179490308
:10AFE0000122D203114308430649086108460021A3
:10AFF0000269082000F077FA002005B0F0BD0000DB
:10B000008CB90008580100200428000034B9000859
:10B0100002000020200000203CB900085CB90008B4
:10B0200068B900086CB900084110000054B9000864
:10B030002200002038B504460D460848808B0443A2
:10B04000224600212C2000F03DFA00956B4601229B
:10B0500006212C2000F05CFA38BD000058010020C9
:10B0600010B5FFF771FC10BD70B505460421362000
:10B0700000F008F90446002D03D00120C00204436B
:10B0800004E00121C90220468843044622460421E7
:10B09000362000F028FA70BDF0B585B006460420D1
:10B0A000029000270020019066494875086300213E
:10B0B00064482030417101730020624988834863ED
:10B0C000886300F0F9F85F49086003E000F0F4F8E5
:10B0D0005C4908605B4800685B498842F6D1002003
:10B0E000FFF764FC59480078432802DD43205749A4
:10B0F000087056480078002802DA0020534908708A
:10B1000052480078242804DD504800780446243C46
:10B110000DE006214D480078FAF700F80621081ADC
:10B1200045014A480078F9F7F9FF2C460C43200600
:10B1300021040843210208432043039000211E20DC
:10B14000039A00F0D0F902AB01220021242000F084
:10B15000DFF91E20FFF7B2FC87B238123949887335
:10B160000420FFF7ABFC01900198C0B200280FD07B
:10B17000022000906B46012212212D2000F0C8F918
:10B180003048808B0121090308432E49888300BF82
:10B1900000F092F82B4908600620FFF78FFC294940
:10B1A00048600720FFF78AFC26498860F806C00E31
:10B1B00008750846007D002801D110200875214936
:10B1C000087D00F0FDF9F007C00F002809D0FFF757
:10B1D0005CFC1C48808B0121C90208431949888303
:10B1E0000CE00521362000F035F8054618480540EA
:10B1F0002A460521362000F065F900BF0120FFF73F
:10B20000D5FB0021042000F03DF80E4988610021A3
:10B21000262000F037F8054605208003054380000E
:10B2200005432A460021262000F05DF90022262150
:10B23000362000F047F900F03FF80249086000208E
:10B2400005B0F0BD580100203001CADE0100002029
:10B25000FFFD0000F8B504460D46094FA9B2A0B2A3
:10B260006B46022200F02EF80646002E06D16846F4
:10B270004078010268460078081887B23846F8BD61
:10B28000FFFF0000FEB505460E460027FF43B1B2A2
:10B29000A8B201AB042200F015F800900098002835
:10B2A00008D1032404E0380201A9095D4718641E8F
:10B2B000002CF8DA3846FEBD10B500210846FFF72D
:10B2C000E1FF10BDFFB581B006460C4617460025CC
:10B2D000002C04D129466D1C684646541AE04020D3
:10B2E0003043C2B229466D1C684642547F2C04DCB0
:10B2F00028466D1C69460C540CE0E0B280210843DE
:10B3000029466D1C6A4650546004020E28466D1C86
:10B3100069460A54A8B23A466946049B00F0AAFA64
:10B3200005B0F0BD70B504460D46164623462A46C4
:10B3300031461120FFF7C6FF70BD10B50446234605
:10B34000052200211520FFF7BDFF10BD10B50446F2
:10B350002346052200211720FFF7B4FF10BD10B5CA
:10B360000446224601210A2000F0BDF810BD70B548
:10B37000054600211A20FFF785FF0446240D240509
:10B380002803000B0443224600211A2000F0ABF8EA
:10B3900070BD000010B50446224602492E2000F080
:10B3A00091F810BD0418000038B504466B46012220
:10B3B00003210420FFF786FF002C16DD2246002122
:10B3C0000C2000F07FF869460878102108430090AF
:10B3D0000F488069090608430D4988616B460122C0
:10B3E0000321042000F094F810E069460878102149
:10B3F00088430090064880690906884304498861AB
:10B400006B4601220321042000F082F838BD0000C1
:10B410005801002010B5044622460021182000F0F3
:10B4200051F810BDF8B50446002500200090002614
:10B430000220204000280AD0802000906B46012284
:10B4400000210D2000F064F801211D480173E00780
:10B45000C00F002826D069460878062108430090CE
:10B460006B46012200210D2000F052F803210F202D
:10B47000FFF7F0FE06468120C0003040002801D1D1
:10B4800000251AE0402000906B46012200210D208B
:10B4900000F03EF80020FFF7E7FD002108480173A7
:10B4A0004D1E0AE0694608780221084300906B4669
:10B4B000012200210D2000F02BF82846F8BD0000E5
:10B4C00078010020F8B505460E461446684604701B
:10B4D00021124170B1B2A8B26B46022200F018F8F6
:10B4E00007463846F8BDFEB506460F461446002509
:10B4F00003E069464C55240A6D1C042DF9DBB9B2F2
:10B50000B0B26B46042200F003F801900198FEBD32
:10B51000FFB581B006460C4617460025002C07D122
:10B5200080203043C2B229466D1C6846425419E05F
:10B53000C0203043C2B228466D1C69460A547F2C95
:10B5400003DC28466D1C0C540CE0E0B2802108435B
:10B5500029466D1C6A4650546004020E28466D1C34
:10B5600069460A54A8B23A466946049B00F0BCF901
:10B5700005B0F0BD70B504460E46154628190121E8
:10B580008902884202DD0020C04370BDA21E3346FE
:10B5900029460920FFF7BCFF0020F6E770B50446F6
:10B5A0000D46064800692043A90508430646324671
:10B5B00000210820FFF797FF002070BD58010020F0
:10B5C00038B504466B4601220E212B20FFF77AFE88
:10B5D00068460078410949010091E106C90E6846B4
:10B5E0000078014300916B4601220E212B20FFF7CA
:10B5F0008FFF38BD70B50146002006E00A541E06D4
:10B60000140A34431B0A2246401C0428F6DB70BD92
:10B6100013B50C4601231A4669460248FDF72EF978
:10B6200000981CBD101A00207CB500210C460D4668
:10B630006846FFF782FE042608E0220E2802104327
:10B64000240205466846805D0443761E002EF4DA27
:10B65000204629467CBD7CB500210C460D46684637
:10B66000FFF774FE042608E0220E2802104324028D
:10B6700005466846805D0443761E002EF4DA2046B7
:10B6800029467CBDFBF73AFBFEF79AF8FDF7B6FCBE
:10B69000FDF792FDFDF7E2FDFDF7B6FDFDF74CFC71
:10B6A000FDF792FCFDF748FEFDF712FBFAF7BCFA36
:10B6B000FAF77CFA0721FF204130FFF7BBFCFFF7C8
:10B6C000CFFC012028490880012201030520000742
:10B6D000FBF7FFFA46E025480078002840D0FEF747
:10B6E0006FF8002021490870FAF734FC20490870EF
:10B6F000084600780F280FDD0122D103052000073E
:10B70000FBF7E7FAFEF7EEF800220121C903052056
:10B710000007FBF7DEFA0BE0012208211548FBF7D2
:10B72000D8FAFEF7DFF8002208211248FBF7D1FA19
:10B73000FDF738FA0C480088002804DD0A48008824
:10B74000401E094908800C48007800280AD10648A4
:10B750000088002806D101210846FBF721FD01E001
:10B76000FDF720FAB7E7000040010020E6000020C6
:10B7700042010020000400504500002000B585B0C3
:10B780001748FBF746FB14216846F9F724FD1548D6
:10B7900000900320019000200290694605200007D8
:10B7A000FBF798F969461048FBF794F969460F488A
:10B7B000FBF790F901210846FBF7F2FCFF2001306E
:10B7C000FBF7C0FC0A4800680421084308490860E8
:10B7D0008815FBF7C9FCFBF7CFFC05B000BD0000E6
:10B7E00088190020FFFF00000004005000080050EE
:10B7F0000070004010B50122D2021B491B48FAF725
:10B800008AFA194800881A4988422CD008461649F5
:10B810000880042088807D20C000C8800120088125
:10B82000002048811E20C04388810120C88100205B
:10B830000884088248828882C882088388834320DB
:10B84000C886012008877820488701208887C88714
:10B850000021054840300184418481840020024950
:10B86000C88300F027F810BD840D002000F0000808
:10B87000AA550000F8B504460F4615461E4600209E
:10B88000009010200521090788620A2322463946C4
:10B890000748FCF7ABFBAAB20A2331460448FCF781
:10B8A000DFFA10200521090788610020F8BD00009B
:10B8B000B819002010B5002472B60121C902084849
:10B8C000FAF70EFA0446002C06D00122D2020549EE
:10B8D0000348FAF7F7FA044662B6204610BD0000A6
:10B8E00000F00008840D0020F8B504460F46154608
:10B8F0001E460020009010200521090788620A23B7
:10B90000224639460948FCF771FB09490870AAB27A
:10B910000A2331460548FCF769FB054908701020E9
:10B920000521090788610020F8BD0000B819002032
:10B93000250000200000010203040005405C000017
:10B94000A05C0400C06C0800805C0400E03F1E00A6
:10B95000E07D1E0007A9022570889B880A0016005A
:10B96000010006000100020087008D002D001A3141
:10B9700052001A339A001A351D011A376B003B31F9
:10B98000BE003B335E013B3596023B3700009959C0
:10B990009959EB518F421E45142E0080EB51F5282A
:10B9A0003333E13A703DE13AC235852BC23533334A
:10B9B000C235C235AE47E13A5138A33051380000A4
:10B9C000000000000000010203040607080900004F
:10B9D000000001020304030406080C1018203000C4
:10B9E00000BA000800000020580100001C5A00089E
:10B9F00038BA000858010020E01D00003AA90008EC
:10BA000021130704380D091E0805400826091040B7
:10BA100008560A131D043B08BE0596D8BC40100802
:10BA2000042FC8420114020214150909010202ADD3
:08BA300081092EE7B15220004C
:04000005080050C1DE
:00000001FF
